:030000000219FDE5
:03000B000200A848
:03002B000201606F
:03005B000202DFBF
:030073000202C5C1
:1000800002030406080C10182030406080040608A3
:100090000C10182030406080A0C000070F1F3F05E3
:1000A000050D050205030302C2AFC0D0C0E0206207
:1000B00017E5256002E473E525F4F58A758B00D217
:1000C00062D0E0D0D0D2AF3285268AC262E526F473
:1000D0006030758B00D0E0D0D0C295C294C293D26C
:1000E000AF32C295C294C293206E0D20660A740589
:1000F000D5E0FDE57EF45290758B00D0E0D0D0D2F3
:10010000AF32758A00C28DD26201F801B73068053E
:10011000206602D29501B7306805206602D29401AC
:10012000B7306805206602D29301B7D29230680AD0
:100130002066077403D5E0FDD29501B7D2913068EF
:100140000A2066077403D5E0FDD29401B7D290D29D
:100150009230680A2066077403D5E0FDD29301B798
:10016000C2AFC2AD53E6EFC0D0C0E0D2D3D2AFC26F
:10017000CEE52A6007207449152A21C1780079004C
:1001800020742EE580307E01F430E70278FF53DAE8
:10019000CF207E0343DA20307E0343DA10C2D8C278
:1001A00071E580307E01F430E70279FFC3E8997091
:1001B000CB306103752A18207403752A18885FD222
:1001C0007020740DE52B6004152B21D143DA01C298
:1001D000D82070024133A85F206102C270207431C0
:1001E000C3E894F0400374F0F8E8C4540F28F87999
:1001F00084B703024111C313C3138721200802C32C
:1002000013200A06C3C898F8411128F8500374FF58
:10021000F8C3E895685003E568F88822E52D540690
:100220006011E533C313C31324062522F5225003BE
:100230007522FF852224A824C3E52495644002A8E2
:10024000648825E56970024177C3E8AA699A50037A
:10025000E8FAE4F9EAC333FBE56BF45B29400D25CA
:100260006AF8E56A6002156A400B41770AC3E56ADD
:100270009A5002056A78FF8826C3E525944040021B
:10028000D26420CF0AD0E0D0D043E610D2AD32C243
:10029000CF053A7801E52A6005307402152AC3E5D6
:1002A0005F9401400575620041BB756300756C0089
:1002B000E5622401F56250037562FFD0E0D0D043BF
:1002C000E610D2AD32C2AFC0D053E67FC2607591A6
:1002D00000855694855795759104D0D0D2AF32C21F
:1002E000AF53E6EFC2ADC0D0C0E0C0F0D2D3D2AFC2
:1002F000A8FBA9FCC2D8307102614653DACF207E38
:100300000343DA10307E0343DA20D271E580307E79
:1003100001F420E702611D88278928A16D53DACFF7
:10032000207E0343DA20307E0343DA10C2D8C27144
:10033000307402A1597800E580307E01F430E70284
:10034000A159885FA14153DACF207E0343DA2030E0
:100350007E0343DA10C271206102811F53DACF207D
:100360007E0343DA10307E0343DA20C2D8D271888C
:100370005A895BC3E89558F8E99559F97B007E08DE
:100380007A00C3E8948CE994005005755E008111F1
:10039000882178A2E6A8216055C3E894C8E99400B2
:1003A0005008E4D2E4FB7A0A61ECC3E89468E9946B
:1003B000015008E4D2E3FB7A0F61ECC3E894D0E982
:1003C00094025008E4D2E2FB7A1E61ECC3E894A0E8
:1003D000E994055008E4D2E1FB7A3C61ECC3E8946F
:1003E00098E994085008E4D2E0FB7A787E00C3E8EC
:1003F000955CFCE9955DFD30E70AECF42401FCED29
:10040000F43400FD755E00C3EC9AED9E5003755EFA
:1004100001885C895D855A58855B597802A141C382
:10042000E89527F8E99528F9307C02A125307B0270
:10043000A125307A02A11E2075028142E9FDE8FC67
:100440008161E9C313F9E813F8307902A11EE9C309
:1004500013F9E813F8307802A11EE9C313FDE8137D
:10046000FC206126C3EC941CED940240028178EDDF
:0F0470007018C3EC94C850120529C3E529940AEB
:10047F005002A159755F00D270A159E5296002158C
:10048F00297888E6F97400207F087896B9030278F6
:10049F009EE624FAFEE43400FFC3EC9EFCED9FFDC4
:1004AF009208B90310A2085007207609D27681C4AA
:1004BF00307602C276A2085016B9030DECF424016F
:1004CF00FCEDF43400FD0204DE78007900A125B9BB
:1004DF000315EC33FCED33FDC3EC940AFCED9400F3
:1004EF00FD50047C007D00C3EC94FFED94004006AA
:1004FF0078FF7900A125EC8575F0A4C5F0A2F7333C
:10050F00F87900400302054178FF7900020541E9BF
:10051F00C313F9E813F8307C0EE9600278FFC3E8E3
:10052F001338F8E43400F9C3E894FFE9940040026B
:10053F0078FF885FD270206102A159741FF4552F84
:10054F004BF52FC274EB7002D274752A18307403F6
:10055F00752A0A306102A16D20740353DAFE2074EC
:10056F0003752B06D0F0D0E0D0D0D2AD43E61032D9
:10057F00790102059D790302059D790A02059D798E
:10058F001E02059D796402059D79C802059D7817A5
:10059F00E4D5E0FDD8FAD9F6227A147B780205C4A7
:1005AF007A107B8C0205C47A0D7BB40205C47A0BDA
:1005BF007BC80205C47902B27DE4D291D5E0FDD2A9
:1005CF0094D5E0FDC294D5E0FDC291D5E0FDD29562
:1005DF00E576D5E0FDC2957496D5E0FDD9D9EAF858
:1005EF00D5E0FDD8FBDBCED29122C37C007D007518
:1005FF00F00005F0EA33FAEB33FB50F6EB13FBEAAE
:10060F0013FAC3E9FFE8FEE89AF8E99BF95004EF03
:10061F00F9EEF8B3EC33FCED33FDD5F0DFEDF9EC8B
:10062F00F822E889F08A20D2D4F8A9F07B0030F7BD
:10063F000B7BFFF42401F8E9F43400F9E88520F08E
:10064F00A4ADF0F8E98520F0A4AFF0FEED2EF9741B
:10065F00003FFA7C04C3EA13FAE913F9E813F8DC54
:10066F00F48BF030F70AE8F42401F8E9F43400F9D8
:10067F00E889F0C2D4F8A9F02222C3E54113F9E5C5
:10068F004013F8C3E54598F8E54699F9500CC3E8CF
:10069F009480E994FF40160206C0C3E8947FE99462
:1006AF000050030206C0787F79000206C078807977
:1006BF00FF884A894B22E54A2547F8E54B3548F92B
:1006CF00854B20E4300701F43549FA30E709C3EAD6
:1006DF0094F040150206FEC3EA940F50030206FE83
:1006EF0078FF79FF7A0F0206FE780079007AF0C35F
:1006FF00E5249564500AC374019524500B02071C1E
:10070F00E54B20E70E02071CE54B30E706884789CB
:10071F00488A492278A4E6FAC3E54A33F8E54B3311
:10072F00F9D131E930E70BC3E89480E994FF401326
:10073F00E156C3E8947FE994005002E156787F793F
:10074F0000E156788079FFE820E715C3E52398F894
:10075F004009C3E89401400302077D780102077D39
:10076F00E8F424012523F8400302077D78FF884C25
:10077F002278A5E6FAA848A949D131E930E70CC398
:10078F00E89401E994FF40160207B1C3E894FFE92A
:10079F00940050030207B178FF79000207B1780186
:1007AF0079FFE920E715C3E54C98F84009C3E894B1
:1007BF000140030207D878010207D8E8F424012585
:1007CF004CF840030207D878FF88242278FFC264D0
:1007DF0020693D206A12D264C3E541940A4009C3DF
:1007EF00E52594405002C26479A1E76023E541609A
:1007FF001F74FF8541F0848539F0306A0375F00569
:10080F00A4F8C5F0600278FFC3E895675002A867A7
:10081F00886622C3E5409440E5419401E5665003A4
:10082F00140133046002F5662202083B2275E8903A
:10083F00227883E6FFE5E820ECF7A8BDA9BE057393
:10084F00C3E57394084052757300E9FA79A0E76025
:10085F0044EA7007E574601B020876C3E89574607C
:0E086F0010E5745006600C140208820460F953
:10087D00020882E574F574C3946D401B7564C0C3A2
:10088D0094044013756480C39404400B756440C395
:10089D009404400375640075BB0622E564F46002A0
:1008AD000564E573B4070375BB1022743279A6870E
:1008BD00F0A4C5F0A2F733F8C3E895644002A8642C
:1008CD0088228824882588268867227540007541EE
:1008DD00F022C2AF75C820A8CCA9CDAA3A30CF015D
:1008ED000A75C824D2AFAB3BAC3C883B893CC3E80E
:1008FD009BF8E99C206908F930670221F42151AD7C
:10090D003D8A3DF9EA9DFA600478FF79FFAE3EAF6E
:10091D003F8B3E8C3FC3EC9FFCC3E99CF542A83B4B
:10092D00A93CC3E89EF8E99FF9C3E54113FBE540F7
:10093D0013FAE82AF540E93BF54150067540FF757D
:10094D0041FF219BAA40AB41AC40AD417E047F02EB
:10095D00C3EB940440021E1FC3EB940840021E1FFC
:10096D00C3ED13FDEC13FCDEF7C3EA9CFAEB9DFB24
:10097D00EF6009C3E913F9E813F8DFF7EA28FAEB9A
:10098D0039FB8A408B4150067BFF8B408B41C3EB7B
:10099D0094025002D2673069047F0321C67892E633
:1009AD00FFC3E537948240110FC3E53794A0400192
:1009BD000FC3EF940640027F057E04E541C4540F3A
:1009CD00F9E541C454F0F8E540C4540F28F8C3E8E4
:1009DD009EFAE99400FB4009C3EA9402EB9400509F
:1009ED00047A02E4FB4140AA40AB41EBC4FEEAC4E9
:1009FD00540F4EFCC3EA9CFAEB9400FBC3E813C3FF
:100A0D0013F8EA28FAEB3400FB8A408B41C3EB94D0
:100A1D00024002C2677804EBC4FE7B00EAC4540FA7
:100A2D004EFAC3EA98FA4005C3940250027A02784E
:100A3D0092E6FF3060024140855256855357D26091
:100A4D0043E680C3E49AF8E49BF930670241DAE8A3
:100A5D00FAE9FBD3E913FDE813FC88528953C3EF80
:100A6D0094036038EF20E00DE82CF8E93DF9ECFA3D
:100A7D00EDFB020A95E828F8E939F9C3E82402F8F4
:100A8D00E93400F97AFE7BFFC3EF9403400E8A54DC
:100A9D008B55884E894F8C508D51610E88548955D8
:100AAD008A4E8B4F8C508D51306920C3E5339403A2
:100ABD004019E542A2E713F8E555F4240138400B3F
:100ACD0020E7087554FFF42401F555610EE8FAD3BB
:100ADD00E813FC8852C3EF94036020EF20E007E891
:100AED002CF8ECFA41FAE8282402F87AFEC3EF94C8
:100AFD000340088A54884E8C50610E88548A4E8C5F
:100B0D0050E56BC3335002646BF56B3060026118B6
:100B1D00753402D26043E680E52D54066026A84068
:100B2D00A941C3E913F9E813F8C2AF53E67F7591F4
:100B3D0000C3E498F594E499F595759104D260435A
:100B4D00E680D2AF22D265754400752000306B036C
:100B5D00752040020B71D265754400752040306BD5
:100B6D0003752000D2AF7801206722E52D54066071
:100B7D0002C265C3E541940540137802940540080F
:100B8D007803940540027806306902780A206019CE
:100B9D00E544601530690AC3E53394034003D53449
:100BAD0006D2AFD26C81427120D2AF0000C2AF200D
:100BBD006726E541C3FB940F40027B0FEB24053004
:100BCD00730123306A02742820620123F93069020F
:100BDD007982E58BC39940B50544E59B5440B5201A
:100BED0002812C30690A08C3E8940A400108619A11
:100BFD002065026171C26553E67F75910030671003
:100C0D007594007595FE759104D26043E68061710F
:100C1D00AE40AF41C3E49EF594E49FF5958113C3B7
:100C2D00E5339402500261713065026171D8028121
:100C3D0040619AC26C53E67F759100855494855539
:100C4D0095759104854E56854F57D26043E680D2F7
:100C5D00AFE52D54066008206A020533020C7C3086
:0F0C6D006C0D206B0A206507158115810214FBA1
:100C7C002278003064053065027801E53775F0079D
:100C8C00A4F9E5F028F5F0E9A2F013A2F113A2F211
:100C9C0013F537C394785003753778C3E537953817
:100CAC004008D266C295C294C29330600281B68568
:100CBC005056855157D26043E68022207D11C2AF39
:100CCC00754302D291C292D2AF759F11020E9EC291
:100CDC00AF754302D291C290D2AF759F11020E9E96
:100CEC00307245207D22C2AF75430390013C757E66
:100CFC0002C293D290D292306204D294A10CC291CF
:100D0C00D2AF759F01020E9EC2AF75430390013C9A
:100D1C00757E02C295D292306204D294A12CC291FB
:100D2C00D2AF759F21020E9E207D17C2AF75430373
:100D3C00900117C293306202D294D2AF759F010218
:100D4C000E9EC2AF754303900117C295306202D25A
:100D5C0094D2AF759F21020E9E207D11C2AF7543B8
:100D6C0004D292C290D2AF759F21020E9EC2AF7573
:100D7C004304D290D292C292D2AF759F01020E9EC2
:100D8C00307243207D20C2AF75430590012B757ED8
:100D9C0004C294D291306204D295A1AAC292D2AF6D
:100DAC00759F11020E9EC2AF75430590014D757E65
:100DBC0001C294D291306204D293A1CAC290D2AF34
:100DCC00759F11020E9E207D17C2AF7543059001D1
:100DDC000DC294306202D295D2AF759F11020E9E55
:100DEC00C2AF754305900121C2943062EBD293D20D
:100DFC00AF759F11020E9E207D13C2AF754306D2B4
:100E0C0090D292C291D2AF759F01020E9EC2AF7565
:100E1C004306D292C291D2AF759F21020E9E3072C0
:100E2C0044207D20C2AF75430190014D757E01C2F7
:100E3C0095D292306204D293C148C290D2AF759FC2
:100E4C0021020E9EC2AF75430190012B757E04C228
:100E5C0093D290D292306204D295C16AC292D2AF30
:100E6C00759F01C19E207D16C2AF75430190012173
:100E7C00C295306202D293D2AF759F21C19EC2AF90
:100E8C0075430190010DC293306202D295D2AF75B9
:100E9C009F01C2662290010B757E00C295C294C25E
:100EAC0093D292D291D290C26222788076FF087649
:100EBC00FF0876FF0876FF08760308760408760AA2
:100ECC00087601087601087601788C76010876FFA1
:100EDC000876FF0876FF0876FF0876FF0876030889
:100EEC0076FF0876FF0876FF0876250876D0087618
:100EFC00FA0876FA0876040876FF08760108760078
:100F0C0008767A0876FF08760108760108760008DC
:100F1C007603227887E6FFC2727888E6C394036072
:100F2C0008C27DE630E102D27DC27E7889E630E1EE
:100F3C0002D27EC3EF94026008758E01D273020F49
:100F4C0052758E00C273227880E6149000809378DC
:100F5C00A4F67881E6149000809378A5F67886E65E
:100F6C001490008D9378A6F6789CE67538FF753949
:100F7C000CB402067538A075390AB40306753882AC
:100F8C0075390578A3E61490009A93F569D1A122DE
:100F9C00227896E6FA7897E6FB7888E6B40305C3E0
:100FAC00EB940EFB307F047A007BFFC3EB9AFCC3FF
:100FBC00948250027C827575000575EC8575F0A4E1
:100FCC00C3E5F0947D40F222D27FF19D12058E7A1A
:100FDC00007B007C10120584E55F2AFA74003BFB51
:100FEC00DCF37C04C3EB13FBEA13FADCF7FEC27FE1
:100FFC00F19D22E5EF20E6037520000520903FFFD0
:10100C00E520146006901DFF1460009304600375C6
:10101C00EF1253D9BF7581C043FF8012057F75EF66
:10102C000243B203E5B3240420E70DF521E5E320E8
:10103C00E0068521B343E301120EA17580FF75A470
:10104C000075F19075D47F75908775A5BF75F2BF4B
:10105C0075D50075A60175E241E4F8F6D8FD756BFF
:0E106C0001120EB612153D7898867675300189
:10107A00C2AF1205981205A812058E1205AF120505
:10108A008E1205B612058E1216561205981205987A
:10109A00120593C2AF78FA79FA308707D9FBD8F7E5
:1010AA00021C00120F1F120F53120F9C120F9D7871
:1010BA00988676120EA175885075891275C824759E
:1010CA00910475D84075A82275B80275E690759B8B
:1010DA0080759D0075D10E75BC5875BB0675BA1121
:1010EA0075E88012057FD2AF12083853DACF207E16
:1010FA000343DA20307E0343DA1043DA01C2D8C24E
:10110A0071120598D2617B037A0CE55E70077A0C3E
:10111A00DB0302109D12058E20700302109DC2701F
:10112A00E55FC3940240E1E52F541F856160F561D4
:10113A00B560D5DAD5C26153DACF207E0343DA200F
:10114A00307E0343DA10C2D8C27178A2E67008D2A0
:10115A0074E52F54E0F52FC27575290012059330F6
:10116A007409C3E529940A4002D2751205847802EB
:10117A003074027800C3E55F9840F0C2AF1205A848
:10118A001205A81205A8D2AF120598754D007888E5
:10119A00E6B40302417D120584788CE6C3940150BB
:1011AA000302127DE530C39401500302127D2074BC
:1011BA0035C3E55F94FF500302127DC2AF1205BD2D
:1011CA00D2AF120593C3E55F940150EFC2AF120587
:1011DA00A81205891205A8D2AF120593C3E55F9438
:1011EA00FF40E90216DB7F05D27F120F9D1205939D
:1011FA00C2AFC27F120F9DAE5FC3E55F947FD2AFCD
:10120A00407B12057FC2AF1205BDD2AFDFDA120FE3
:10121A00D4C3EE94057897F612059812157F121624
:10122A005E7F0AD27F120F9D120593C2AFC27F1250
:10123A000F9DAE5FC3E55F947FD2AF50E412057F86
:10124A00C2AF1205A81205891205A8D2AFDFD412BF
:10125A000FD4EE24057896F612059812157F121609
:10126A008D120593120F9DC3E55F94FF500221B8BA
:10127A000216DBC3E55F954D4003855F4D1205936A
:10128A0078017988E7B403027805C3E55F984002DC
:10129A002198C2AF1205BD1205BD1205BDD2AF120B
:1012AA000598753000E4F531F5320531E531F47011
:1012BA00390532789AE67819146012783214600D7A
:1012CA00787D14600878FA146003753200C3E53239
:1012DA0098401715327531B478998676C2AF1205DF
:1012EA00BDD2AF78988676120593120589E52A70E1
:1012FA0005307402019D78012074027806C3E55F07
:10130A009840A77888E6C394036003120593E52AF8
:10131A00700302109DC2AF120EA1E4F522F523F567
:10132A0024F525F526F56AD2AF7885E6C333F56844
:10133A00E4F545F546F547F548F549F573F52CF515
:10134A002DF53775730875BB1012057F12083CE539
:10135A00E820ECFBA8BDA9BEE97001F88874120860
:10136A004075730875BB107887E6FE7602120F1F68
:10137A007887EEF6C2AF7564FF1208B885226485D5
:10138A002265852266D2AF75220175240175250171
:10139A0075260185636C756D017888E6B40307C20A
:1013AA007D307602D27DD268D269753300120E037F
:1013BA00120E2A1208D81208DF1208D81208DF12F1
:1013CA0008D80213DCC2AF120F1FD2AF75730075B3
:1013DA00BB06120B63120688120C7D120CC7120888
:1013EA00DF120B52306D031206892067031207DBE6
:1013FA00306703120822120C7D120CEC1208DF125D
:10140A000B63306D031206C5120C7D120D651208AE
:10141A00DF120B52306D03120723120C7D120D8C52
:10142A001208DF120B63306D03120780120C7D1253
:10143A000E031208DF12083C120B52120C7D120E18
:10144A002A1208401208DF306932206B2F85676440
:10145A0085676585636C756D0179187A0CC3E53308
:0F146A0099400CC269D26A8A357564FF021486F4
:10147900C3E55F940140030213DC021503306A1BC4
:10148900206B18E535147004C26A61CFF535C3E5E0
:101499005F940140030213DC021503753600C3E5AE
:1014A900627882985054307404E52A604D7888E651
:1014B900B40317207D0520760781D330760281D3C6
:1014C900206B07D26B856764811B78F0306B0585CB
:1014D90067647820C3E54198500261DC306B1BC218
:1014E9006BC27D307602D27DD26A7535128567640A
:1014F90061DC0536E55F6002A106753600C2AF12F0
:101509000EA17887E6FE7602120F1F7887EEF6E4C1
:10151900F522F523F524F525F526F568C268D2AF3D
:1015290012057F120EA1307409C3E53694054002F5
:10153900019D41AF901A0D78201215C1E520B45ACA
:101549000CA31215C1E520B4A50302155F120EB64E
:1015590012157F02157E901A0378807B0A1215C135
:10156900A308DBF9901A0F788C7B181215C1A30810
:10157900DBF9901A2722C2AF1216001215DA901A57
:1015890000740E1215C6A374041215C6A37414129E
:1015990015C6901A0378807B0A1215C5A308DBF9D2
:1015A900901A0F788C7B181215C5A308DBF912164F
:1015B900131215F1901A2722E493F622E6438F01BC
:1015C900538FFD75EF0275B7A575B7F1F0538FFE0F
:1015D90022438F02438F0175EF0275B7A575B7F1E5
:1015E900901A0DF0538FFC22901A0D745AB1C690BF
:1015F9001A0E74A5B1C6227A3079D07820901A4093
:10160900B1C1E520F709A3DAF7227A3079D0901A27
:1016190040E7B1C609A3DAF922AB77A878BB010282
:101629007984BB02027985BB03027986BB040279FE
:1016390092BB05027987BB060279A3BB0702799C95
:10164900BB08027988BB09027989E8F7227C05126F
:101659000598DCFB22C2AF1205A81205AF1205B628
:101669001205BD1205891205A81205AF1205B61299
:1016790005BD1205891205A81205AF1205B6120596
:10168900BDD2AF22C2AF1205BD1205B61205AF1207
:1016990005A81205891205BD1205B61205AF120576
:1016A900A81205891205BD1205B61205AF1205A8C3
:1016B900D2AF22AE77AF78C2AF1205A81205A81231
:1016C90005A8120589DEF21205BD120589DFF8D2D7
:1016D900AF22D15ED156D1567577017578017579EA
:1016E90000D1BC7C05AD5F120598C3ED955F70F51F
:1016F900C3E55F9401400AC3E55F94FF40320217D6
:1017090017D122B17FD15EC2AF75EF12D156DCD5A8
:101719000579C3E5799403500280C6D1560578E569
:10172900771490009F93F808C3E57898500280AE2B
:10173900D156D1560577C3E577940A5002809C1299
:0B1749000EB6B17FC2AF75EF12D15693
:0319FD00020FFFD7
:101A00000E0414FFFFFFFF03040A0101015AA501A0
:101A1000FFFFFFFFFF03FFFFFF25D0FAFA04FF01DE
:081A2000007AFF01010003FF41
:101A400023585032354123202020202020202020E0
:101A500023424C48454C4923463333302320202031
:101A60002020202020202020202020202020202076
:101C0000C2AFC2D353D9BF7581C043B20343FF8073
:101C1000752438752503B1C975EF0275E24043F1AB
:101C20008053A47F75D400D2877DFA780379E67C4F
:101C300010752200752300901DD67B0675249875BB
:101C400025013087028142208708D8FBD9F9DCF7CB
:101C500081B4308708D8FBD9F9DCF781B4B189E4C5
:101C600093A3C39A6004DDC381B4DBDBB17B600264
:101C7000812B7B08E493FAA3B15CDBF87A30B15C8A
:101C8000752200752300B17BEAFCEBFDC3ED94FEE9
:101C9000400EB17B8A278B28ED30E0048A828B834B
:101CA000B17B7AC270D8C3ED94FE601350CEBD00F4
:101CB00025EC60097520007521FF0200008100A855
:101CC00027A9280809D804D90281D3B17FEA89AAB3
:101CD000F281C50D81A0C3ED94035049EDA2E092BD
:101CE000007AC5C3E5829400E583941C50902000DF
:101CF00010438F02438F0175B7A575B7F1F030001F
:101D00001FA827A9280809438F01538FFDD804D99C
:101D100002A12089AAE275B7A575B7F1F0A3A10DBC
:101D2000538FFC817C7AC1BD030CE493A3FAB140CC
:101D3000DCF8B138817C817EAA22AB23B15CEBFA5E
:101D4000EA6222752608C3E52313F523E52213F57D
:101D50002250066323A0632201D526EAB1C9B1C986
:101D600075260AEAF4200102D287300102C287B147
:101D7000C9C3134002C201D526EB22B17FEAFB2082
:101D80008702A17F308702A184752608AE24AF2583
:101D9000C3EF13FFEE13FEB1CDB1C9C3EA13308711
:101DA000024480FA30E703632201C3E52313F523DD
:101DB000E52213F52250066323A0632201D526D91C
:101DC000E52265236523F52222AE24AF250E0FDE22
:101DD000FEDFFCD20122424C48656C693437316326
:041DE000F3300601D5
:00000001FF
